:020000000C945E
:1000020048040C9400000C9400000C9400000C9422
:1000120000000C94E7040C9400000C94CD040C94A2
:1000220000000C9400000C9400000C9400000C944E
:10003200AD180C9400000C9400000C9400000C9479
:1000420000000C9400000C947A040C9400000C94B0
:1000520000000C9400000C9400000C9400000C941E
:1000620000000C9400000C9400000C9400000C940E
:1000720000000C9400000C9400000C9400000C94FE
:1000820000000C9400000C9400001027E8036400A8
:100092000A000100001000011000010020202020B1
:1000A20020CFD0CECFD3D1D2C8D2DC202020202066
:1000B20000002020202020CDC0D1D2D0CEC8D2DC5A
:1000C20020202020202000002020202020CFD0CE61
:1000D200CFD3D1D2C8D2DC20202020200000202083
:1000E200202020CDC0D1D2D0CEC8D2DC20202020EA
:1000F200202000002020202020CFD0CECFD3D1D26C
:10010200C8D2DC202020202000002020202020CD6A
:10011200C0D1D2D0CEC8D2DC2020202020200000A6
:100122002020202020CFD0CECFD3D1D2C8D2DC20E5
:100132002020202000002020202020CDC0D1D2D09D
:10014200CEC8D2DC20202020202000002020202029
:10015200202020202020202020202020202020209D
:1001620000202020CFD0CED6C5D1D120D0C0C1CE44
:10017200D2DB2020200020202020CDCEC2C0DF20D4
:10018200CFC0C9CAC0202020200020CFD0CEC4CEEC
:10019200CBC6C5CDC8C520CFC0C9CAC82020002043
:1001A2002020C4CECF2E20CDC0D1D2D0CEC9CAC835
:1001B20020202000C2CDC5D8CDC5C520CFCEC4CA0F
:1001C200CBDED7C5CDC8C52000202020202ACFCE27
:1001D200C4CACBDED7C5CDCE2A20202020002020C5
:1001E2002ACDC520CFCEC4CACBDED7C5CDCE2A20DC
:1001F20020200020202020D0C5C6C8CC20D0C0C1DD
:10020200CED2DB2020202000202020202020D1D28E
:10021200C0CDD6C8DF2020202020202000C2C5D09B
:10022200D5CDC8C920CDC0C3D0C5C2C0D2C5CBDCD4
:1002320000202020CFCEC4CEC3D0C5C220CFCBC099
:10024200D2DB202020002020202020D0C5C1CECB10
:10025200CBC8CDC320202020200020202020D0D3B6
:10026200D7CDCEC920D0C5C6C8CC202020200020A2
:100272002020CFD0CED4C8CBDC20CFC0C9CAC82062
:10028200202020002020202020536E36332F506261
:100292003337202020202020002020202020202052
:1002A20020536E4167202020202020202000202083
:1002B200202020CFD0CED4C8CBDC2030202020205C
:1002C2002020002020202020CFD0CED4C8CBDC207C
:1002D20031202020202020002020202020CFD0CE1E
:1002E200D4C8CBDC20322020202020200020202057
:1002F2002020CFD0CED4C8CBDC2033202020202019
:1003020020002020202020CFD0CED4C8CBDC203427
:10031200202020202020002020202020CFD0CED43A
:10032200C8CBDC20352020202020200020CFD0CEBA
:10033200D4C8CBDC20CFCEC4CEC3D0C5C2C020200F
:1003420000202020CFD0CED4C8CBDC20C2C5D0D54F
:10035200C0202020200020CFD0CED4C8CBDC20D09B
:10036200C5C1CECBCBC8CDC3C0200020CDC0D1D219
:10037200D0CEC9CAC020CFD0CED4C8CBDF20200077
:1003820020202054552B253475B0432020200020F6
:10039200202020CCC5D1D2C020CFC0C9CAC82020BD
:1003A2002020200020202020D2C5CCCFC5D0C0D212
:1003B200D3D0C02020202020002020202020204B2D
:1003C2003D253275202020202020202000C2C5D0CB
:1003D200D5CDC5C3CE20CDC0C3D0C5C2C0D2C5CB3A
:1003E200DF002020202020CA2DCFD0CED4C8CBDFE2
:1003F200202020202020002020204D41583D253360
:100402007520002020202020CCCED9CDCED1D2DC28
:1004120020202020202000CDC8C6CDC5C3CE20CDAF
:10042200C0C3D0C5C2C0D2C5CBDF002020205057E8
:1004320020253475202020002020202020CCCED959
:10044200CDCED1D2DC2020202020002020202AC2A4
:10045200D0C5CCDF20CFC0C9CAC82A2020202000A6
:100462005425337520D1C5CA202020205425327549
:1004720020D7C0D12000202020204D41583D2533D7
:100482007520202020202020200020202020202035
:10049200CCCED9CDCED1D2DC2020202020200020ED
:1004A20020D2C5CCCFC5D0C0D2D3D0C020C2CACBF7
:1004B2002E20200020202020202054454D5025337E
:1004C200752020200020202020202020CFCBC0D249
:1004D200DB202020202020202000D2C5CCCFC5D078
:1004E200C0D2D3D0C020CDC0C3D0C5C2C00020204E
:1004F20020D0C5C6C8CC20CACECDD2D0CECBDF202C
:1005020020200020202020202AC2CACBDED7C5CD41
:100512002A2020202020200020202020202AC2DB88
:10052200CACBDED7C5CD2A20202020200020D4D35C
:10053200CDCAD6C8DF20C4CECDC0C3D0C5C2C0206C
:1005420020002020202020C4CECDC0C3D0C5C2C0F0
:1005520020202020202000202020D2C5CCCF2EC455
:10056200CECDC0C3D0C5C2C0202020002020202074
:1005720020E2E5F0F1E8FF20332E34202020202075
:1005820000202020C4CECFCECBCDC8D2C5CBDCCD6F
:10059200DBC5202020002020202020CDC0D1D2D0B9
:1005A200CEC9CAC820202020202000202020202AB6
:1005B200CFD0CECFD3D1D2C8D2DC2A202020200067
:1005C200202AC4C0D2D7C8CA20312028C2C5D0D55B
:1005D200292A2020002AC4C0D2D7C8CA2032202803
:1005E200CDC8C6CDC8C9292A2000202020CFD0C519
:1005F200C420D3D1D2C0CDCEC2CAC8202020002070
:100602002020202020DFD0CACED1D2DC2020202002
:100612002020200020202020205455253375202022
:100622002020202000202020202054442533752023
:10063200202020202000202020202020205455256A
:100642003375202020202020202000202020202060
:10065200D3D1D2C0CDCEC2C8D2DC202020202000EF
:100662002020CDC0D7C0D2DC20D0C0C1CED2D32072
:10067200CFCE202000C7C0C4C0CDCDDBCC20D3D18B
:10068200D2C0CDCEC2CAC0CC00205444253375B0EE
:10069200432C20205455253375B043002054442563
:1006A2003375B04300202020CDC0D7C0D2DC20D08B
:1006B200C0C1CED2D320202020002020C220D0D3FF
:1006C200D7CDCECC20D0C5C6C8CCC5202020005462
:1006D2003D2025750A4700533D2025750A53004EDB
:1006E2003D2025750A57004B3D2025750A560050BE
:1006F2003D332E340A52004C3D2025750A68004FC6
:100702003D73740A5300473D73740A5300523DD13E
:10071200F2E0EDF6E8FF0A5700523DC2C5D0D50A15
:100722005700523DCFEEE4EEE3F0E5E20A57005205
:100732003DD0E5E1EEEBEBE8EDE30A5700523DD0A8
:10074200F3F7EDEEE90A5700503D536E36332F5062
:100752006233370A5700503D536E41670A570050C3
:100762003DCFF0EEF4E8EBFC20300A5700503DCFCD
:10077200F0EEF4E8EBFC20310A5700503DCFF0EEEA
:10078200F4E8EBFC20320A5700503DCFF0EEF4E8DB
:10079200EBFC20330A5700503DCFF0EEF4E8EBFCBF
:1007A20020340A5700503DCFF0EEF4E8EBFC203540
:1007B2000A5700503DCDE5F20A5700D1D2C0CDD63E
:1007C200C8DF202000C2C5D0D5202020202000CFA5
:1007D200CEC4CEC3D0C5C22000D0C5C1CECBCBC8FB
:1007E200CDC30020536E36332F50623337002020A2
:1007F20020202020536E416700CFD0CED4C8CBDC5E
:10080200203000CFD0CED4C8CBDC203100CFD0CE28
:10081200D4C8CBDC203200CFD0CED4C8CBDC20333E
:1008220000CFD0CED4C8CBDC203400CFD0CED4C8B9
:10083200CBDC20350048C8C7202020202A42504562
:100842004DDF2A20204245505820200050572533A2
:100852007520202A2534752A20205057253375000B
:1008620074253375B0432074253375B04320742545
:100872003375B043000080C001002D4E414E000090
:10088200020081057808010088057A080000F894C2
:10089200EE27ECBBF1E0F5BFE5BFE0936C00F8E1B9
:1008A200F1BDE1BD8DE0A2E0BB27ED938A95E9F7AA
:1008B20080E090E1A0E0B1E0ED930197E9F7E2E892
:1008C200F8E085919591009761F0A591B591059019
:1008D2001590BF01F00105900D920197E1F7FB0120
:1008E200F0CFEFEFEDBFE0E1EEBFC0E0D5E00C945A
:1008F200001C0E940C241A930A931BB10CB1A12F65
:10090200B0E0ECE1F0E0EA23FB233097E1F4E09180
:100912007E05F0E0E45BFA4F0083A0917E05AF5FB5
:10092200A0937E05A23319F4E0E0E0937E05A09146
:100932008005AF5FA0938005A23329F4E0E0E09345
:100942008005689420F80E941A24E03019F405D03A
:10095200E0934905099119912BC01A93E091800502
:10096200E030E1F3E0917F05F0E0E45BFA4F1081C3
:10097200A0917F05AF5FA0937F05A23319F4E0E059
:10098200E0937F05F894E0918005E150E0938005C3
:100992007894E12F199108950E940C240E941F243B
:1009A2000E9426240E942D240E9434240E943B246B
:1009B200E991EFBFF991E991B991A9919991899141
:1009C20079916991F9901990099018950E940C24D7
:1009D2000E943F21989B4FC00E946D240E94722466
:1009E2000E947B240E948024E3E6F1E00E9484249A
:1009F2000E948824999B04C00E948E240E94932402
:100A0200999902C0A895FCCF0E9498249A9B04C091
:100A12000E948E240E949E249A9902C0A895FCCF1F
:100A22000E9498240E948E24E33028F0A0E0B0E0D7
:100A3200E0E00E94A82C0E948E240E94A32429F4A4
:100A42000E948824E8E7F1E011C0E130A0E0FA0753
:100A520029F40E948824ECE8F1E008C0E230A0E02A
:100A6200FA0741F40E948824E1EAF1E0FA93EA935A
:100A72000E948B21AFCF0E94A6240E948E24E230D6
:100A820010F00C948A05989B42C00E94AE240E94EA
:100A920080240E94B1240E946D24E6EBF1E00E94C2
:100AA2008424999B04C00E941A240E949324999939
:100AB20002C0A895FCCF0E9498249A9B04C00E9471
:100AC2001A240E949E249A9902C0A895FCCF0E94E3
:100AD20098240E941A24E23028F0A9E2B1E0E0E072
:100AE2000E94A82C0E941A24E03031F40E9488242B
:100AF200EBECF1E00E9484240E941A24E13031F4EC
:100B02000E948824E0EEF1E00E948424BCCF0E947F
:100B1200A6240E948E24E23010F00C94E905989BE2
:100B220055C00E946D240E9472240E947B240E9460
:100B32008024E5EFF1E00E948424999B03C0F30135
:100B420031973F01999902C0A895FCCF0E94982441
:100B52009A9B03C0F30131963F019A9902C0A8956E
:100B6200FCCF0E9498240E94B42410F466247724B7
:100B7200062C072831F40E948824EAE0F2E00E9461
:100B820084240E94B92431F40E948824EFE1F2E027
:100B92000E9484240E94BE2431F40E948824E3E34C
:100BA200F2E00E9484240E94C32431F40E9488242B
:100BB200E8E4F2E00E9484240E94B42431F40E940A
:100BC2008824ECE5F2E00E948424A9CF0E94A624A6
:100BD2000E948E24E23010F00C94FA06062C0728AC
:100BE20011F00C94FA06989B02C10E946D240E9497
:100BF20072240E947B240E948024E1E7F2E00E949A
:100C0200842499994A94999902C0A895FCCF0E948C
:100C120098249A9943949A9902C0A895FCCF0E946D
:100C22009824E7E0E41508F444244420C1F40E9427
:100C320088240E94C8240E94CB24A2E6B0E00E942D
:100C4200F4240E94FB24A8E3B0E00E940425AAE356
:100C5200B0E00E940B250E9412250E941D25E1E0B2
:100C6200E415C1F40E9488240E9424250E942725AD
:100C7200A4E6B0E00E94F4240E945025A2E4B0E071
:100C82000E940425A4E4B0E00E940B250E9459258D
:100C92000E941D25E2E0E415C1F40E9488240E940E
:100CA20064250E946725A6E6B0E00E94F4240E9413
:100CB2009025ACE4B0E00E940425AEE4B0E00E94CE
:100CC2000B250E9499250E941D25E3E0E415D1F42D
:100CD2000E948824E5ECF2E00E9484240E94A4256C
:100CE200A2E7B0E00E94F4240E94CD25A6E7B0E07E
:100CF2000E940425A8E7B0E00E940B250E94D62599
:100D02000E941D25E4E0E415D1F40E948824EAED56
:100D1200F2E00E9484240E94E125A4E8B0E00E944F
:100D2200F4240E940A26A8E8B0E00E940425AAE85A
:100D3200B0E00E940B250E9413260E941D25E5E0CB
:100D4200E415D1F40E948824EFEEF2E00E9484249C
:100D52000E941E26A6E9B0E00E94F4240E944726C3
:100D6200AAE9B0E00E940425ACE9B0E00E940B259C
:100D72000E9450260E941D25E6E0E415D1F40E944F
:100D82008824E4E0F3E00E9484240E945B26A8EA1F
:100D9200B0E00E94F4240E948426ACEAB0E00E94F3
:100DA2000425AEEAB0E00E940B250E948D260E9427
:100DB2001D25E7E0E415D1F40E948824E9E1F3E07F
:100DC2000E9484240E949826AAEBB0E00E94F42498
:100DD2000E94C126AEEBB0E00E940425A0ECB0E078
:100DE2000E940B250E94CA260E941D25FCCE0E944D
:100DF200D5260E948E24E23010F00C945A070E94ED
:100E0200BE2411F00C945A070E943F21989B4DC0BA
:100E12000E946D240E9472240E947B240E948024DE
:100E2200EEE2F3E00E94842499998A94999902C08F
:100E3200A895FCCF0E9498249A9983949A9902C00B
:100E4200A895FCCF0E949824E2E0E81508F48824D3
:100E5200882061F40E9488240E94C8240E94DD2612
:100E62000E94F026A4ECB0E00E94F726E1E0E8152B
:100E720061F40E9488240E9424250E94FF260E9479
:100E8200F026ABECB0E00E94F726E2E0E81561F450
:100E92000E9488240E9464250E9412270E94F02644
:100EA200A2EDB0E00E94F726B1CF0E9425270E9452
:100EB2003F210E948E24E23010F00C94B4070E946D
:100EC200B92411F00C94B4070E943F21989B49C0A9
:100ED2000E946D240E9472240E947B240E9480241E
:100EE200E3E4F3E00E9484249999DA94999902C088
:100EF200A895FCCF0E9498249A99D3949A9902C0FB
:100F0200A895FCCF0E949824E2E0ED1508F4DD24B8
:100F1200DD2041F40E9488240E94C8240E942B27CD
:100F22000E943627E1E0ED1561F40E9488240E94B8
:100F32002425ABEDB0E00E943D27ADEDB0E00E946C
:100F42003627E2E0ED1561F40E9488240E946425B0
:100F5200AFEDB0E00E943D27A1EEB0E00E9436273F
:100F6200B5CF0E94D5260E948E24E23010F00C9458
:100F720042080E94C32411F00C9442080E943F21AF
:100F8200989B7DC00E946D240E9472240E947B2443
:100F92000E948024E8E5F3E00E9484249999CA948F
:100FA200999902C0A895FCCF0E9498249A99C3945B
:100FB2009A9902C0A895FCCF0E949824E4E0EC150F
:100FC20008F4CC24CC2051F40E9488240E94C82426
:100FD2000E944427A9EEB0E00E944F27E1E0EC1501
:100FE20081F40E9488240E942425ABEDB0E00E9487
:100FF2005627ADEEB0E00E94F026AFEEB0E00E94C0
:101002004F27E2E0EC1581F40E9488240E946425B7
:10101200A3EFB0E00E945627A3EFB0E00E94F026B3
:10102200A5EFB0E00E944F27E3E0EC1591F40E9497
:101032008824E5ECF2E00E948424A9EFB0E00E944B
:101042005627A9EFB0E00E94F026ABEFB0E00E9475
:101052004F27E4E0EC1591F40E948824EAEDF2E0D7
:101062000E948424AFEFB0E00E945627AFEFB0E0B9
:101072000E94F026A1E0B1E00E944F2781CF0E949A
:10108200D5260E948E24E23010F00C949808062C8B
:10109200072811F00C949808989B47C00E946D2471
:1010A2000E9472240E947B240E9480240E945D2759
:1010B2000E9488240E946027999B04C00E94662790
:1010C2000E946B27999902C0A895FCCF0E94982490
:1010D2009A9B04C00E9466270E9470279A9902C0B8
:1010E200A895FCCF0E9498240E946627329720F090
:1010F200A6E0B0E00E9475270E946627309741F46F
:101102000E947A27EEE9F0E00E944A2E0E947F2791
:101112000E946627319741F40E947A27E4EBF0E0BF
:101122000E944A2E0E947F27B7CF0E94A6240E94C7
:101132008E24E23010F00C94EF080E94BE2411F0CD
:101142000C94EF08989B48C00E946D240E94722460
:101152000E947B240E9480240E945D270E94882492
:101162000E946027999B04C00E9486270E949324B4
:10117200999902C0A895FCCF0E9498249A9B04C01A
:101182000E9486270E949E249A9902C0A895FCCFAD
:101192000E9498240E948627E23028F0A1E0B0E065
:1011A200E0E00E94A82C0E948627E03041F40E94D1
:1011B2007A27EAECF0E00E944A2E0E947F270E94E2
:1011C2008627E13041F40E947A27E0EEF0E00E94A7
:1011D2004A2E0E947F27B6CF0E94A6240E948E2408
:1011E200E23010F00C9446090E94B92411F00C94DC
:1011F2004609989B48C00E946D240E9472240E9456
:101202007B240E9480240E945D270E9488240E94E1
:101212006027999B04C00E948B270E94932499996E
:1012220002C0A895FCCF0E9498249A9B04C00E94F9
:101232008B270E949E249A9902C0A895FCCF0E94F7
:1012420098240E948B27E23028F0A2E0B0E0E0E090
:101252000E94A82C0E948B27E03041F40E947A273A
:10126200E6EFF0E00E944A2E0E947F270E948B2721
:10127200E13041F40E947A27ECE0F1E00E944A2E2C
:101282000E947F27B6CF0E94A6240E948E24E230BD
:1012920010F00C949D090E94C32411F00C949D0936
:1012A200989B48C00E946D240E9472240E947B2455
:1012B2000E9480240E945D270E9488240E94602749
:1012C200999B04C00E9490270E949324999902C07E
:1012D200A895FCCF0E9498249A9B04C00E94902754
:1012E2000E949E249A9902C0A895FCCF0E9498243D
:1012F2000E949027E23028F0A3E0B0E0E0E00E94F4
:10130200A82C0E949027E03041F40E947A27E2E262
:10131200F1E00E944A2E0E947F270E949027E1302E
:1013220041F40E947A27E8E3F1E00E944A2E0E94EB
:101332007F27B6CF0E94A6240E948E24E23010F0AE
:101342000C94210A062C072811F00C94210A989B70
:101352006BC00E9488240E94B1240E9495270E949B
:101362009A270E94B1270E94B6270E946D240E94EC
:10137200B927999B04C00E94BC270E94C1279A9B4F
:1013820004C00E94BC270E94CA270E94D32710F0E3
:101392000E941F24E42D0E94A32429F40E94DB272B
:1013A200A2E3B0E03EC0E130A0E0FA0729F40E94D7
:1013B200DB27ACE3B0E035C0E230A0E0FA0729F465
:1013C2000E94DB27A6E4B0E02CC0E330A0E0FA07DD
:1013D20029F40E94DB27A8E6B0E023C0E430A0E0B5
:1013E200FA0729F40E94DB27AAE7B0E01AC0E53029
:1013F200A0E0FA0729F40E94DB27ACE8B0E011C0B4
:10140200E630A0E0FA0729F40E94DB27AEE9B0E05B
:1014120008C0E730A0E0FA0731F40E94DB27A0EB16
:10142200B0E00E94A02C93CF0E94BE2411F40E942F
:1014320034240E94BE2411F40E941F240E94A62478
:101442000E948E24E23010F00C94780A0E94B92493
:1014520011F00C94780A989B3EC00E9488240E9446
:10146200B1240E9495270E949A270E94B1270E94C8
:10147200B6270E946D240E94B927999B04C00E943E
:10148200BC270E94C1279A9B04C00E94BC270E94CD
:10149200CA270E94D32710F00E941F24ED2D0E941C
:1014A200A32429F40E94DB27A7EDB0E011C0E130AC
:1014B200A0E0FA0729F40E94DB27ABEDB0E008C0F8
:1014C200E230A0E0FA0731F40E94DB27AFEDB0E092
:1014D2000E94A02CC0CF0E94BE2411F40E9434248A
:1014E2000E94BE2411F40E941F240E94A6240E947E
:1014F2008E24E230D0F50E94B424B9F5989B33C013
:101502000E9488240E94B1240E9495270E94E0270D
:101512000E94E5270E94EA270E94B1270E94B6276F
:101522000E946D240E94B927999B06C00E94E5275C
:101532000E946B270E94F9279A9B06C00E94E5270A
:101542000E9470270E94F9270E94E527ED32A1E050
:10155200FA0720F0A3E0B1E00E947527A3E0B1E012
:101562000E943D27CBCF0E94A6240E948E24E23007
:1015720010F00C94410B062C072811F00C94410B2F
:101582000E946627319711F00C94410B989B76C00C
:101592000E9488240E94B1240E9495270E94FF275E
:1015A2000E94B1270E9408280E946D240E940B28E5
:1015B200999B06C00E940E280E946B270E94F92761
:1015C2009A9B06C00E940E280E9470270E94F9274B
:1015D2000E940E28B49710F00E9413280E940E2831
:1015E2003F9710F40E941328E42D0E94A32429F4AB
:1015F2000E940E28A6E5B0E03EC0E130A0E0FA0766
:1016020029F40E940E28A8E5B0E035C0E230A0E03F
:10161200FA0729F40E940E28AAE5B0E02CC0E330B4
:10162200A0E0FA0729F40E940E28AEE6B0E023C03B
:10163200E430A0E0FA0729F40E940E28A0E8B0E006
:101642001AC0E530A0E0FA0729F40E940E28A2E9A8
:10165200B0E011C0E630A0E0FA0729F40E940E289B
:10166200A4EAB0E008C0E730A0E0FA0731F40E9433
:101672000E28A6EBB0E00E94A02C88CF0E94A624E0
:101682000E948E24E23010F00C94D80B062C07280E
:1016920011F00C94D80B0E946627319711F00C942C
:1016A200D80B989B82C00E9488240E94B1240E9479
:1016B2009527E9EFF3E0FA93EA930E941A280E9431
:1016C2001F280E94B1270E9408280E946D24E5E08D
:1016D200F4E00E948424999B04C0A7E3B5E00E9431
:1016E2002E289A9B04C0A7E3B5E00E943128A0915E
:1016F2003705B0913805A436E0E0BE0714F00E9429
:101702003428A0913805AA2332F4E0E0F0E0E09317
:101712003705F0933805E42D0E94A32429F40E9492
:101722001A28A5E0B1E03EC0E130A0E0FA0729F4B2
:101732000E941A28A7E0B1E035C0E230A0E0FA0723
:1017420029F40E941A28A9E0B1E02CC0E330A0E0FD
:10175200FA0729F40E941A28ABE0B1E023C0E43072
:10176200A0E0FA0729F40E941A28ADE0B1E01AC0FD
:10177200E530A0E0FA0729F40E941A28AFE0B1E0B0
:1017820011C0E630A0E0FA0729F40E941A28A1E16C
:10179200B1E008C0E730A0E0FA0731F40E941A284D
:1017A200A3E1B1E00E94A02C7CCF0E94A6240E945B
:1017B2008E24E23010F00C94360C0E94B92411F001
:1017C2000C94360C0E948B27E13011F00C94360CED
:1017D200989B49C00E9488240E94B1240E949527A8
:1017E2000E94FF270E94B1270E9408280E946D24B0
:1017F2000E940B28999B06C00E940E280E946B270C
:101802000E94F9279A9B06C00E940E280E94702708
:101812000E94F9270E940E28B49710F00E94132804
:101822000E940E283F9710F40E941328ED2D0E946B
:10183200A32429F40E940E28A9EDB0E011C0E130E2
:10184200A0E0FA0729F40E940E28ADEDB0E008C02E
:10185200E230A0E0FA0731F40E940E28A1EEB0E0D7
:101862000E94A02CB5CF0E94A6240E948E24E230B2
:1018720010F00C94C00C062C072811F00C94C00C2C
:101882000E946627319711F00C94C00C989B6BC094
:101892000E9488240E94B1240E9495270E94E0277A
:1018A2000E943B280E94EA270E94B1270E944028FA
:1018B2000E946D240E94B927999B02C00E9443286E
:1018C2009A9B02C00E9446280E94492810F00E945A
:1018D2002624E42D0E94A32429F40E943B28A4E399
:1018E200B0E03EC0E130A0E0FA0729F40E943B28B4
:1018F200AEE3B0E035C0E230A0E0FA0729F40E947E
:101902003B28A8E4B0E02CC0E330A0E0FA0729F4B9
:101912000E943B28AAE6B0E023C0E430A0E0FA0728
:1019220029F40E943B28ACE7B0E01AC0E530A0E001
:10193200FA0729F40E943B28AEE8B0E011C0E63075
:10194200A0E0FA0729F40E943B28A0EAB0E008C010
:10195200E730A0E0FA0731F40E943B28A2EBB0E0A6
:101962000E94A02C93CF0E94B92411F40E942D242E
:101972000E94B92411F40E9426240E94A6240E94E7
:101982008E24E23010F00C941D0D0E94BE2411F042
:101992000C941D0D0E948627E13011F00C941D0D50
:1019A200989B3EC00E9488240E94B1240E949527E1
:1019B2000E94E0270E943B280E94EA270E94B1274A
:1019C2000E9440280E946D240E94B927999B02C060
:1019D2000E9443289A9B02C00E9446280E944928DE
:1019E20010F00E942624E82D0E94A32429F40E94CC
:1019F2003B28A2ECB0E011C0E130A0E0FA0729F4E4
:101A02000E943B28A9ECB0E008C0E230A0E0FA074F
:101A120031F40E943B28A0EDB0E00E94A02CC0CF80
:101A22000E94B92411F40E942D240E94B92411F4B9
:101A32000E9426240E94A6240E948E24E23010F0E6
:101A42000C94850D0E94C32411F00C94850D0E9404
:101A52009027E13011F00C94850D989B53C00E94A1
:101A620088240E94B1240E9495270E94E0270E94A8
:101A72003B280E94EA270E94B1270E9440280E9428
:101A82006D240E94B927999B02C00E9443289A9B09
:101A920002C00E9446280E945128A732E2E0BE07F7
:101AA20010F00E942624EC2D0E94A32429F40E9407
:101AB2003B28A5EEB0E023C0E130A0E0FA0729F40C
:101AC2000E943B28ABEEB0E01AC0E230A0E0FA0779
:101AD20029F40E943B28A1EFB0E011C0E330A0E05E
:101AE200FA0729F40E943B28A7EFB0E008C0E430CF
:101AF200A0E0FA0731F40E943B28ADEFB0E00E946B
:101B0200A02CABCF0E94A6240E948E24E23010F0BB
:101B12000C94050E0E94C32411F00C94050E0E9431
:101B22009027E13011F00C94050E989B6BC00E9437
:101B320088240E94B1240E949527EDE2F4E0FA93F2
:101B4200EA930E9456280E941F280E94B1270E94F1
:101B520008280E946D24EAE3F4E00E948424999B01
:101B620006C00E9456280E946B270E94F9279A9B62
:101B720006C00E9456280E9470270E94F9270E94E0
:101B82005628E536A0E0FA0724F0A3EEB0E00E9462
:101B92005B28A4EEB0E00E948C2CEE2322F4A3EE8C
:101BA200B0E00E947527EC2D0E94A32429F40E9424
:101BB2005628A9EEB0E023C0E130A0E0FA0729F4EC
:101BC2000E945628AFEEB0E01AC0E230A0E0FA0759
:101BD20029F40E945628A5EFB0E011C0E330A0E03E
:101BE200FA0729F40E945628ABEFB0E008C0E430AF
:101BF200A0E0FA0731F40E945628A1E0B1E00E9469
:101C0200A02C93CF0E94A6240E948E24E23010F0D2
:101C12000C94BF0E0E94C32411F00C94BF0E0E94BC
:101C22009027E13011F00C94BD0E989BA5C00E9444
:101C320060280E9472240E9463280E94B1240E949C
:101C42006D24EDE4F4E00E9484240E949527E2E6EC
:101C5200F4E0FA93EA93E0911F05F09120050E94C7
:101C62006728E0911D05F0911E050E9467280E94D9
:101C72006C280E9488240E9495270E947E21999BAD
:101C82001AC00E94F9270E94712831976040704063
:101C92000E94982CEF5FFF4F6F4F7F4FAFE1B5E08F
:101CA2000E9476280E947C2830F40E948428E093C7
:101CB2001F05F09320059A9B11C00E94F9270E94EC
:101CC2007128EF5FFF4F6F4F7F4F0E94982C319723
:101CD20060407040AFE1B5E00E948D28A0911F05E1
:101CE200B0912005A43FE1E0BE0760F0A6E1B0E0BC
:101CF200E4EFF1E060E070E00E94982CE0931F05B1
:101D0200F09320059B9B13C00E94F9270E94712823
:101D1200E051FE40604070400E9493280E94762865
:101D22000E947C2820F40E9484280E949A28CF9B3B
:101D320022C00E94F9270E947128E05FF14F6F4F85
:101D42007F4F0E9493280E948D280E947128E038BC
:101D5200A1E5FA07A1E06A07A0E07A0760F0A6E130
:101D6200B0E0E0E8F1E561E070E00E94982CE8E183
:101D7200F0E00E949A2859CF0E94A6240E948E2445
:101D8200E23010F00C944A0F062C072811F00C9444
:101D92004A0F0E946627319711F00C944A0F989BC4
:101DA20076C00E9488240E94B1240E9495270E9436
:101DB2009F280E94B1270E9440280E946D240E9401
:101DC2000B28999B06C00E94A8280E946B270E949C
:101DD200AD289A9B06C00E94A8280E9470270E94E4
:101DE200AD280E94A828B49710F00E94B3280E9440
:101DF200A8283F9710F40E94B328E42D0E94A32440
:101E020029F40E94A828ACE5B0E03EC0E130A0E091
:101E1200FA0729F40E94A828AEE5B0E035C0E23006
:101E2200A0E0FA0729F40E94A828A0E6B0E02CC09E
:101E3200E330A0E0FA0729F40E94A828A0E7B0E066
:101E420023C0E430A0E0FA0729F40E94A828A2E8FF
:101E5200B0E01AC0E530A0E0FA0729F40E94A828F1
:101E6200A4E9B0E011C0E630A0E0FA0729F40E942C
:101E7200A828A6EAB0E008C0E730A0E0FA0731F4EB
:101E82000E94A828A8EBB0E00E94A02C88CF0E9454
:101E9200A6240E948E24E23010F00C94E10F062C4E
:101EA200072811F00C94E10F0E946627319711F078
:101EB2000C94E10F989B82C00E9488240E94B12456
:101EC2000E949527E8E7F4E0FA93EA930E94BA2881
:101ED2000E941F280E94B1270E9440280E946D2460
:101EE200ECE8F4E00E948424999B04C0A9E3B5E0E5
:101EF2000E942E289A9B04C0A9E3B5E00E943128D3
:101F0200A0913905B0913A05A436E0E0BE0714F07D
:101F12000E94BF28A0913A05AA2332F4E0E0F0E043
:101F2200E0933905F0933A05E42D0E94A32429F4A5
:101F32000E94BA28A5E1B1E03EC0E130A0E0FA0774
:101F420029F40E94BA28A7E1B1E035C0E230A0E04E
:101F5200FA0729F40E94BA28A9E1B1E02CC0E330C3
:101F6200A0E0FA0729F40E94BA28ABE1B1E023C04D
:101F7200E430A0E0FA0729F40E94BA28ADE1B1E00A
:101F82001AC0E530A0E0FA0729F40E94BA28AFE1AE
:101F9200B1E011C0E630A0E0FA0729F40E94BA28A5
:101FA200A1E2B1E008C0E730A0E0FA0731F40E94F4
:101FB200BA28A3E2B1E00E94A02C7CCF0E94A62402
:101FC2000E948E24E23010F00C943F100E94BE2436
:101FD20011F00C943F100E948627E13011F00C940E
:101FE2003F10989B49C00E9488240E94B1240E94FD
:101FF20095270E949F280E94B1270E9440280E9494
:102002006D240E940B28999B06C00E94A8280E945A
:102012006B270E94AD289A9B06C00E94A8280E94A6
:1020220070270E94AD280E94A828B49710F00E9441
:10203200B3280E94A8283F9710F40E94B328E82DE5
:102042000E94A32429F40E94A828A7ECB0E011C0A2
:10205200E130A0E0FA0729F40E94A828AEECB0E033
:1020620008C0E230A0E0FA0731F40E94A828A5EDEA
:10207200B0E00E94A02CB5CF0E94A6240E948E241C
:10208200E23010F00C94B6100E94C32411F00C94AC
:10209200B6100E949027E13011F00C94B6100E9405
:1020A20051280E94332E10F00C94B610989B5BC0FE
:1020B2000E9488240E94B1240E9495270E949F2892
:1020C2000E94B1270E9440280E946D240E940B2882
:1020D200999B06C00E94A8280E946B270E94AD28E7
:1020E2009A9B06C00E94A8280E9470270E94AD28D1
:1020F2000E94A828B49710F00E94B3280E94A82832
:102102003F9710F40E94B328EC2D0E94A32429F4D7
:102112000E94A828A7EEB0E023C0E130A0E0FA07B1
:1021220029F40E94A828ADEEB0E01AC0E230A0E087
:10213200FA0729F40E94A828A3EFB0E011C0E33007
:10214200A0E0FA0729F40E94A828A9EFB0E008C08D
:10215200E430A0E0FA0731F40E94A828AFEFB0E023
:102162000E94A02CA3CF0E94A6240E948E24E230BB
:1021720010F00C944711062C072811F00C9447110B
:102182000E946627319711F00C944711989B7CC0EE
:102192000E9488240E9472240E9480240E9408289F
:1021A2000E946D24E1EAF4E00E9484240E949527B3
:1021B2000E94C6280E94CF280E9495270E947E2155
:1021C200999B06C00E94D6280E946B270E94F9277D
:1021D2009A9B06C00E94D6280E9470270E94F92767
:1021E2000E94D628EB3FA0E0FA0720F0AEE2B0E072
:1021F2000E947527E42D0E94A32429F40E94D62868
:10220200A0E5B0E03EC0E130A0E0FA0729F40E9468
:10221200D628A2E5B0E035C0E230A0E0FA0729F402
:102222000E94D628A4E5B0E02CC0E330A0E0FA0773
:1022320029F40E94D628ACE6B0E023C0E430A0E046
:10224200FA0729F40E94D628AEE7B0E01AC0E530BA
:10225200A0E0FA0729F40E94D628A0E9B0E011C054
:10226200E630A0E0FA0729F40E94D628A2EAB0E0FC
:1022720008C0E730A0E0FA0731F40E94D628A4EBA8
:10228200B0E00E94A02C82CF0E94A6240E948E243D
:10229200E23010F00C94AD110E94BE2411F00C94A7
:1022A200AD110E948627E13011F00C94AD11989B7C
:1022B20051C00E9488240E9472240E948024E7EC6C
:1022C200F4E00E9484240E946D24ECEDF4E00E946C
:1022D20084240E9495270E94C6280E94CF280E942B
:1022E20095270E947E21999B06C00E94D6280E94B3
:1022F2006B270E94F9279A9B06C00E94D6280E944B
:1023020070270E94F9270E94D628EB3FA0E0FA0727
:1023120020F0AEE2B0E00E947527E82D0E94A324CF
:1023220029F40E94D628A5ECB0E011C0E130A0E06B
:10233200FA0729F40E94D628ACECB0E008C0E230DB
:10234200A0E0FA0731F40E94D628A3EDB0E00E9483
:10235200A02CADCF0E94A6240E948E24E23010F061
:102362000C944612062C072811F00C9446120E9477
:102372006627319711F00C944612989B84C00E94F4
:10238200AE240E9480240E9440280E946D24E0EF27
:10239200F4E00E948424999B04C00E94DB280E94DE
:1023A2006B27999902C0A895FCCF0E9498249A9B0A
:1023B20004C00E94DB280E9470279A9902C0A89547
:1023C200FCCF0E9498240E94DB28329710F00E94D2
:1023D200E0280E94DB28309721F40E9488240E9482
:1023E200E3280E94DB28319721F40E9488240E946E
:1023F200E628E42D0E94A32429F40E94DB28A2E609
:10240200B0E03EC0E130A0E0FA0729F40E94DB28E8
:10241200A4E6B0E035C0E230A0E0FA0729F40E9459
:10242200DB28A6E6B0E02CC0E330A0E0FA0729F4EE
:102432000E94DB28A2E7B0E023C0E430A0E0FA0764
:1024420029F40E94DB28A4E8B0E01AC0E530A0E03D
:10245200FA0729F40E94DB28A6E9B0E011C0E630B1
:10246200A0E0FA0729F40E94DB28A8EAB0E008C03D
:10247200E730A0E0FA0731F40E94DB28AAEBB0E0D3
:102482000E94A02C7ACF0E94A6240E948E24E230C1
:1024920010F00C94B2120E94BE2411F00C94B212ED
:1024A2000E948627E13011F00C94B212989B57C01B
:1024B2000E94AE240E9480240E9440280E946D2423
:1024C200E0EFF4E00E948424999B04C00E94DB2880
:1024D2000E946B27999902C0A895FCCF0E9498246C
:1024E2009A9B04C00E94DB280E9470279A9902C01E
:1024F200A895FCCF0E9498240E94DB28329710F006
:102502000E94E0280E94DB28309721F40E94882450
:102512000E94E3280E94DB28319721F40E9488243C
:102522000E94E628E82D0E94A32429F40E94E928AB
:10253200A4ECB0E011C0E130A0E0FA0729F40E9457
:10254200E928ABECB0E008C0E230A0E0FA0731F4D1
:102552000E94E928A2EDB0E00E94A82CA7CF0E9419
:10256200A6240E948E24E23010F00C944F13062C05
:10257200072811F00C944F130E946627319711F02F
:102582000C944F13989B88C00E94AE240E94802412
:102592000E9440280E946D24EFE2F5E00E9484240C
:1025A200999B04C00E94EE280E946B27999902C051
:1025B200A895FCCF0E9498249A9B04C00E94EE2802
:1025C2000E9470279A9902C0A895FCCF0E94982475
:1025D2000E94EE28329720F0A8E0B0E00E94752712
:1025E2000E94EE28309721F40E9488240E94E3285A
:1025F2000E94EE28319721F40E9488240E94E62846
:10260200E42D0E94A32429F40E94EE28A6E3B0E060
:102612003EC0E130A0E0FA0729F40E94EE28A0E4CF
:10262200B0E035C0E230A0E0FA0729F40E94EE28BB
:10263200AAE4B0E02CC0E330A0E0FA0729F40E943B
:10264200EE28A4E7B0E023C0E430A0E0FA0729F4C2
:102652000E94EE28A6E8B0E01AC0E530A0E0FA0732
:1026620029F40E94EE28A8E9B0E011C0E630A0E00B
:10267200FA0729F40E94EE28AAEAB0E008C0E7307F
:10268200A0E0FA0741F40E94EE28ACEBB0E00E9411
:10269200A02C0E94F32876CF0E94A6240E948E24AA
:1026A200E23010F00C94F013062C072811F00C9471
:1026B200F0130E946627319711F00C94F0130E94D8
:1026C200EE28309711F00C94EE13989B86C00E946E
:1026D20088240E94B1240E943F210E946028E4E4E1
:1026E200F5E00E9484240E946D24E1EAF4E00E9455
:1026F20084240E949527E6EBF4E0FA93EA930E9481
:10270200FA280E9467280E94CF280E9495270E94DB
:102712007E21999B06C00E94FA280E946B270E9484
:10272200F9279A9B06C00E94FA280E9470270E94ED
:10273200F9270E94FA28EB3FA0E0FA0720F0AAE06E
:10274200B0E00E947527E42D0E94A32429F40E9480
:10275200FA28A8E3B0E03EC0E130A0E0FA0729F48D
:102762000E94FA28A2E4B0E035C0E230A0E0FA0705
:1027720029F40E94FA28ACE4B0E02CC0E330A0E0D7
:10278200FA0729F40E94FA28A6E7B0E023C0E43051
:10279200A0E0FA0729F40E94FA28A8E8B0E01AC0DB
:1027A200E530A0E0FA0729F40E94FA28AAE9B0E08D
:1027B20011C0E630A0E0FA0729F40E94FA28ACEA38
:1027C200B0E008C0E730A0E0FA0731F40E94FA282E
:1027D200AEEBB0E00E94A02C78CF0E94A6240E940B
:1027E2008E24E23010F00C949114062C072811F07C
:1027F2000C9491140E946627319711F00C94911455
:102802000E94EE28309711F00C949114989B7CC092
:102812000E943F210E9488240E94B1240E94952791
:102822000E94E0270E94FF280E94EA270E94B12707
:102832000E9440280E946D24E9E5F5E00E9484246C
:10284200999B06C00E94FF280E946B270E94F927CD
:102852009A9B06C00E94FF280E9470270E94F927B7
:102862000E94FF28EB3EA1E0FA0720F0ACE0B0E0C6
:102872000E947527E42D0E94A32429F40E94FF28B8
:10288200AAE3B0E03EC0E130A0E0FA0729F40E94DA
:10289200FF28A4E4B0E035C0E230A0E0FA0729F452
:1028A2000E94FF28AEE4B0E02CC0E330A0E0FA07BB
:1028B20029F40E94FF28A8E7B0E023C0E430A0E09A
:1028C200FA0729F40E94FF28AAE8B0E01AC0E5300E
:1028D200A0E0FA0729F40E94FF28ACE9B0E011C099
:1028E200E630A0E0FA0729F40E94FF28AEEAB0E041
:1028F20008C0E730A0E0FA0731F40E94FF28A0ECFC
:10290200B0E00E94A02C82CF0E94B92411F40E9450
:102912002D240E94B92411F40E9426240E94A62488
:102922000E948E24E23011F00C94CD16989B5CC06C
:102932000E948824EEE6F5E00E9484240E946D2421
:10294200E3E8F5E00E9484240E946028E8E9F5E0CB
:102952000E94842499999A94999902C0A895FCCFCF
:102962000E9498249A9993949A9902C0A895FCCFB0
:102972000E949824E5E0E91508F49924992031F49D
:102982000E940429EDEAF5E00E948424E1E0E915C1
:1029920031F40E940429E2ECF5E00E948424E2E092
:1029A200E91531F40E940429E7EDF5E00E94842440
:1029B200E3E0E91531F40E940429EDE4F4E00E9419
:1029C2008424E4E0E91531F40E940429ECEEF5E0F8
:1029D2000E948424E5E0E91531F40E940429E1E033
:1029E200F6E00E948424A2CF0E942527E1E0E915A7
:1029F20059F5989B29C00E949527E6E1F6E0FA93E3
:102A0200EA930E9407290E9467280E940C290E94CB
:102A120095270E947E21999B06C00E9407290E9449
:102A22006B270E94AD289A9B06C00E9407290E942C
:102A320070270E94AD280E940729F39720F0AAE28E
:102A4200B0E00E947527D5CF0E94AD28E2E0E915DB
:102A520059F5989B29C00E949527E7E2F6E0FA9380
:102A6200EA930E9411290E9467280E940C290E9461
:102A720095270E947E21999B06C00E9411290E94DF
:102A82006B270E94AD289A9B06C00E9411290E94C2
:102A920070270E94AD280E941129F39720F0ACE222
:102AA200B0E00E947527D5CFE3E0E91559F5989B70
:102AB20029C00E949527E8E3F6E0FA93EA930E9480
:102AC20016290E9467280E940C290E9495270E94BD
:102AD2007E21999B06C00E9416290E946B270E94A4
:102AE200AD289A9B06C00E9416290E9470270E9458
:102AF200AD280E941629FD9720F0A4E1B0E00E94C3
:102B02007527D5CFE4E0E91511F00C949B16989B3C
:102B120011C10E948824EDE4F6E00E948424A2E31D
:102B2200B0E0E3ECF0E00E94A02CA4E3B0E00E944D
:102B32001B29A6E3B0E00E942029ACE3B0E0E6EE58
:102B4200F0E00E94A02CAEE3B0E00E941B29A0E4BA
:102B5200B0E00E942029A6E4B0E0E6EEF0E00E9498
:102B6200A02CA8E4B0E00E941B29A0E5B0E0EEE6AC
:102B7200F0E00E94A02CA2E5B0E0E3E7F0E00E94C2
:102B8200A02CA4E5B0E0E9E6F0E00E94A02CA6E5C6
:102B9200B0E00E942529A8E5B0E00E942529AAE517
:102BA200B0E00E942529ACE5B0E00E942529AEE5FF
:102BB200B0E00E942529A0E6B0E00E942529A2E605
:102BC200B0E00E947527A4E6B0E00E947527A6E651
:102BD200B0E00E947527AAE4B0E00E947527ACE439
:102BE200B0E0E2EDF0E00E94A02CAEE4B0E00E9482
:102BF2002A29A4E5B0E00E945B28A6E6B0E00E9484
:102C02007527A2ECB0E0E0E9F1E00E94A02CA4EC70
:102C1200B0E0E0E00E94A82CA5ECB0E0E2E8F0E031
:102C22000E94A02CA7ECB0E0E8E1F0E00E94A02C0A
:102C3200A5EEB0E00E941B29A7EEB0E0E8E1F0E0CB
:102C42000E94A02CA9EEB0E0E0E5F0E00E94A02CEA
:102C5200A0E2B0E0E0EFF0E00E94A02CE0E0F0E0C3
:102C62000E949A28A6E1B0E0E0E0F0E060E070E0C7
:102C72000E94982CA7EDB0E0ECEDF0E00E94A02CB1
:102C8200A9EDB0E0E4E1F0E00E94A02CAAE2B0E0FD
:102C92000E942A29ACE2B0E00E942A29A4E1B0E015
:102CA200EAE0F0E00E94A02C55240E94E028A0E077
:102CB200B0E0E0E00E94A82C662477240E942F292D
:102CC2000E9436290E943B290E943E29A8E0B0E0DA
:102CD2000E942029A2E2B0E00E947527A4E2B0E09F
:102CE2000E947527A6E2B0E00E947527A8E2B0E034
:102CF2000E947527A3E0B1E0E4EBF0E00E94A02C73
:102D02000E94BF280E943428A5E1B1E00E945B28FE
:102D1200A5E0B1E00E945B28A7E1B1E00E945B2838
:102D2200A7E0B1E00E945B28A9E2B1E0E1E00E94E5
:102D3200A82CEDCEE5E0E91559F5989B29C00E9433
:102D42009527E8E3F6E0FA93EA930E9449290E9464
:102D520067280E940C290E9495270E947E21999B38
:102D620006C00E9449290E946B270E94AD289A9BA7
:102D720006C00E9449290E9470270E94AD280E9425
:102D82004929FD9720F0A7E2B1E00E947527D5CF2F
:102D92000E943F210E942527062C072811F00C943F
:102DA2005517A895989B80C00E9488240E94B12440
:102DB2000E946D240E944E290E9460280E9451297F
:102DC2000E9495270E9454290E945A290E946C2829
:102DD2000E9404290E9495270E945C290E943E2994
:102DE2000E94F328E2E3E0931005A895E42D0E94E7
:102DF200A32439F40E94CB240E94FB240E941225B2
:102E02004CC0E130A0E0FA0739F40E9427250E9465
:102E120050250E94592541C0E230A0E0FA0739F45A
:102E22000E9467250E9490250E94992536C0E330B2
:102E3200A0E0FA0739F40E94A4250E94CD250E9441
:102E4200D6252BC0E430A0E0FA0739F40E94E12530
:102E52000E940A260E94132620C0E530A0E0FA074D
:102E620039F40E941E260E9447260E94502615C051
:102E7200E630A0E0FA0739F40E945B260E9484261D
:102E82000E948D260AC0E730A0E0FA0761F40E9492
:102E920098260E94C1260E94CA260E94882CE0938E
:102EA2003705F09338057ECF0E94B92411F00C94B7
:102EB2009717A895989B3AC0A8950E9488240E94CB
:102EC200B1240E946D240E944E290E9460280E9413
:102ED20051290E9495270E9463290E94CF280E94AF
:102EE20095270E945C290E943E290E94F3280E9495
:102EF2002624ED2D0E94A32419F40E942B270EC034
:102F0200E130A0E0FA0721F0E230A0E0FA0761F434
:102F1200ABEDB0E00E943D27ADEDB0E00E94882C01
:102F2200A0E1B0E00E94A02CA895C4CF0E94BE24CC
:102F320011F00C94DE17A895989B3FC0A8950E94AB
:102F420088240E94B1240E946D240E944E290E946E
:102F520060280E9451290E9495270E9454290E94AC
:102F6200D6280E9467280E946C280E9404290E9489
:102F720095270E945C290E943E290E94F3280E9404
:102F82001F24E82D0E94A32419F40E94DD260DC0FF
:102F9200E130A0E0FA0719F40E94FF2606C0E230F1
:102FA200A0E0FA0741F40E9412270E94882CAEE0AA
:102FB200B0E00E94A02CA895BFCF0E94C32411F0BC
:102FC2000C945718A895989B71C0A8950E948824C4
:102FD2000E94B1240E946D240E944E290E94602802
:102FE2000E9451290E949527EEE9F6E0FA93EA93AE
:102FF2000E943B280E9467280E94CF280E949527A2
:103002000E945C29A0E2B0E00E9475270E943E293E
:103012000E94F328A895EC2D0E94A32429F40E9473
:103022004427A9EEB0E03BC0E130A0E0FA0759F432
:10303200ABEEB0E00E945627ADEEB0E00E94F02663
:10304200AFEEB0E02CC0E230A0E0FA0759F4A1EFF5
:10305200B0E00E945627A3EFB0E00E94F026A5EF51
:10306200B0E01DC0E330A0E0FA0759F4A7EFB0E0EA
:103072000E945627A9EFB0E00E94F026ABEFB0E025
:103082000EC0E430A0E0FA0781F4ADEFB0E00E9498
:103092005627AFEFB0E00E94F026A1E0B1E00E9417
:1030A200882CA3EEB0E00E94A02C8DCF0E94B42405
:1030B20021F5A895989B21C0A8950E9488240E947A
:1030C200B1240E946D24E7EAF6E00E9484240E9463
:1030D2006028ECEBF6E00E9484240E9495270E946F
:1030E20063290E94CF280E9495270E945C290E9492
:1030F2003E290E94F328A895DDCF0E948E24E0305D
:10310200E1F4A5E2B1E00E9475270E9468290E94BD
:103112006B29AA24BB240E942F29E0931305F09364
:1031220014050E943B29E0E0F0E00E943629E0E02D
:10313200F0E0E0931505F09316050E948E24E2302C
:1031420041F4A8E0B0E00E9420290E9426240E94B7
:103152001F240E943F21A2C10E940C240E946E29BA
:103162000E943B28EA1BFB0BE0932D05F0932E05F2
:10317200062C0728C1F40E9473292CF00E947A2998
:1031820012F40E942D24A8950E94732964F4A09140
:103192003605AA2312F40E942D240E94872914F0D6
:1031A2000E948F29A8950E94B92411F40E942D240F
:1031B2000E94BE24E1F40E9473292CF00E947A2915
:1031C20012F40E942D240E9473298CF4A0913605DA
:1031D200AA2312F40E942D240E94872914F00E942F
:1031E2008F290E949629E0932705F09328050E94D3
:1031F200C32449F40E945128129728F00E949B2967
:1032020010F00E94A029A0912505B09126050E94E8
:10321200A529EA1BFB0BE0932F05F09330050E94D2
:10322200AA290E94DB27EA1BFB0BE0933105F093EE
:103232003205E1E0E515F9F4A895062C0728D9F442
:103242000E94AF290E94332E5CF40E94AF29159789
:103252003CF40E94B4290E94B9290E94BE29A89573
:103262000E94D42944F4A8950E94D9290E94DE29FB
:1032720012F40E943424E1E0E515E9F4062C072853
:10328200D1F40E94D6280E94E729A8F40E94EB29D3
:103292000E94D62832960E94F02968F40E94B92929
:1032A2000E94332E40F40E94F429E436A0E0FA078B
:1032B20010F40E94F929E1E0E51551F50E94B924C4
:1032C20039F50E94EB290E94D929309711F40E9406
:1032D200022A0E94092A54F40E94AF29159734F455
:1032E2000E94B4290E94B9290E94BE290E94D429B1
:1032F2003CF40E94D9290E94DE2912F40E9434244F
:103302000E940D2AA536E0E0BE0714F00E94122AA0
:103312000E94BE2411F40E9434240E940D2AA43675
:10332200E0E0BE0714F00E94122AE1E0E515D1F4B4
:103332000E94C324B9F40E945128119738F40E94C4
:1033420056280E94192A11F40E94A0290E94562888
:103352000E940D2AAE17BF072CF40E949B2910F47D
:103362000E941D2A0E94202A0E94A529E093250579
:10337200F09326050E94262AE13BA4E0FA0740F0DA
:103382000E9426240E941F240E946B290E943B292E
:10339200E1E0E51581F5E3E0F0E06E167F0658F511
:1033A2000E94D6280E94F02920F00E94F4290E944F
:1033B20070270E94F429DF010E94332EE0F40E945C
:1033C200D628DF010E94332EB0F40E94F429E4369D
:1033D200A0E0FA0780F40E94F9290E94F429EC592E
:1033E200FF4FA0E3B0E00E94A02C0E94DB283097A0
:1033F20011F40E942B2AE1E0E51511F00C944B1A0E
:103402000E94AF29119714F00C944B1AF5013196D2
:103412005F01E2E0F0E06E167F06E0F500240A1498
:103422000B0420F4F501EC59FF4F5F01E6E6F0E0F2
:10343200EA15FB0590F00E94B9290E94332E70F420
:10344200E5E6F0E05F01EA15FB0541F40E94F92987
:103452000E94312AAC9A0E94312AAC980E94162905
:103462000E94372AEA15FB05A8F40E9434240E9420
:103472002D240E941F240E9426240E946B290E9450
:103482003B2955240E943C2A0E943F2A0E943F2A3F
:103492000E944D2A0E94262A0E947027E991EFBFBE
:1034A200F991E991B991A99199918991799169914A
:1034B200F9901990099018951A930A93B89AC09A9C
:1034C2000E94562AC0980E945E2AE0933B05F09320
:1034D2003C058BE18A95F1F70E945E2AE0933F0555
:1034E200F0934005C09AE0913B05F0913C050E94A3
:1034F200642ADF01CB01E0913F05F09140050E9473
:103502006C2AAAE2B0E027C01A930A93A79AAF9A4C
:103512000E94562AAF980E945E2AE0933D05F093DE
:103522003E058BE18A95F1F70E945E2AE093410500
:10353200F0934205AF9AE0913D05F0913E050E945D
:10354200642ADF01CB01E0914105F09142050E941E
:103552006C2AACE2B0E00E94882C0E947A2ADF0139
:10356200CB01E0E0F0E068EC72E40E94EE2DADECFD
:10357200BCEC8CEC9DE30E94522DD8018827992740
:103582000E94742C0E94A02D0E94E62C8F01F8014B
:103592000991199108950E941F240E9426240E94D5
:1035A2002D240E9434240E943B2408950E941A2450
:1035B200E03059F4E1E0E51541F4A0914905A33565
:1035C20021F4E9DFE0E0E09349050E941A24E030AB
:1035D20069F4552059F4A0914905AA3539F4E1E07E
:1035E200E0934A05A0914A05A130E1F3E1EDF6E04E
:1035F200FA93EA930E94A5290E9467280E947F2AD3
:10360200E9EDF6E0FA93EA930E94262A0E946728DF
:103612000E947F2AE1EEF6E00E94842A0E947F2A1D
:10362200E9EEF6E0FA93EA930E948B2A0E947F2A3F
:10363200E1EFF6E00E94902AE9EFF6E0FA93EA93CE
:103642000E9496290E9467280E947F2AE1E0E515E0
:1036520021F4E1E0F7E00E94902A552021F4E8E00D
:10366200F7E00E94902AF301309719F4EFE0F7E0B7
:103672001BC0E130A0E0FA0719F4EBE1F7E014C057
:10368200E230A0E0FA0719F4E4E2F7E00DC0E3301B
:10369200A0E0FA0719F4E1E3F7E006C0E430A0E0A5
:1036A200FA0741F4EFE3F7E0FA93EA9380E00E942D
:1036B200DD232296062C072811F00C94A11BE42D81
:1036C2000E94A32419F40E94972A3AC0E130A0E094
:1036D200FA0719F40E949A2A33C0E230A0E0FA07EE
:1036E20019F40E949D2A2CC0E330A0E0FA0729F4C5
:1036F200EFE6F7E00E94902A23C0E430A0E0FA0748
:1037020029F4EDE7F7E00E94902A1AC0E530A0E024
:10371200FA0729F4EBE8F7E00E94902A11C0E6309C
:10372200A0E0FA0729F4E9E9F7E00E94902A08C02C
:10373200E730A0E0FA0721F4E7EAF7E00E94902AD6
:103742000E94B924A1F4ED2D0E94A32419F40E9431
:10375200972A0DC0E130A0E0FA0719F40E949A2AD4
:1037620006C0E230A0E0FA0711F40E949D2A0E94EE
:10377200BE24A1F4E82D0E94A32419F40E94972AE2
:103782000DC0E130A0E0FA0719F40E949A2A06C09F
:10379200E230A0E0FA0711F40E949D2A0E94C3249D
:1037A20031F5EC2D0E94A32419F40E94972A1FC020
:1037B200E130A0E0FA0719F40E949A2A18C0E23018
:1037C200A0E0FA0719F40E949D2A11C0E330A0E09C
:1037D200FA0729F4EFE6F7E00E94902A08C0E430E5
:1037E200A0E0FA0721F4EDE7F7E00E94902A0E9498
:1037F200B42421F4E5EBF7E00E94902A0895E0E872
:10380200EBBBEABBE0E0E8BBEFEFE7BBEFE6E5BB13
:10381200E0E9E4BBE0E0E2BBE1BBE0E5E3B9E8E01C
:10382200E2B9E0E0E0936200E0936100E0936500BA
:10383200E0936400E0BFE7E6E3BFE0E0E2BFE1BFA0
:10384200EFBDE4E0EEBDE0E0EDBDECBDE7BDE6BD01
:10385200EAE7EBBDE2E1EABDE0E0E9BDE8BDE09305
:103862007900E0937800EBE6E5BDE0E0E4BDE3BD7E
:10387200E1E8E0938B00E5E0E0938A00E0E0E0938A
:103882008900E0938800E0938100E0938000E09358
:103892008700E0938600E0938500E0938400E09344
:1038A2008300E0938200E0936A00EABFE0E5E9BFAB
:1038B200E8BFE0E1E7BFE0E0E0937D00EBB9E8E9D3
:1038C200EAB9E6E0E0939500E0E0E0939000EFE2F1
:1038D200E9B9E0E8E8B9E0E0E0BDE3E5EDB9E0E050
:1038E200EEB9E4E1EA930E94AD21EFE1E1BDEFE040
:1038F200E1BD78940E943F210E946B2966247724BF
:103902000E94F328E1E0E0934905E0E0E0934A05F4
:10391200E1E0E51511F00C94FA1D062C072811F0D0
:103922000C943D1D0E94EE28319751F4A8950E94F7
:10393200A8280E94A02A0E94262A0E94AD2AA895A1
:103942000E94EE28309711F00C94F91C0E94A828CE
:103952000E94A02A0E94B82A319729F4A8950E94B1
:10396200262A0E94AD2A0E94B82A3B9798F0A89571
:10397200AEE1B0E00E94882C0E94AD2A0E94BD2ACE
:10398200EA0FFB1F0E94C32AAEE1B0E00E94882C1E
:103992000E947027E1E0E51559F5A8950E94FA28E2
:1039A2000E94E72928F50E94B82A3197B9F4A89510
:1039B2000E94FF280E945128EA0FFB1FE093230573
:1039C200F09324050E94B82A3A96A4E0B0E00E943F
:1039D200A02CAC9A0E94C82AA895AC980E94DB271A
:1039E2000E94E72928F40E942B2A0E94CE2AA89539
:1039F2000E94BD2AEA17FB0718F4A8950E94CE2A56
:103A02000E947329CCF50E94D02A0E94D52AA8953B
:103A12000E94E32A20F40E94EB2A319603C00E94FE
:103A2200EB2A3197FE93EE93A895A0911C05AA2349
:103A320012F40E94F02A0E94F72A14F00E94FF2A30
:103A4200A0913605AA2312F40E942D240E94BA28BE
:103A52003197A0913505B0913605EA17FB0734F48A
:103A62000E94BA28E0933505F09336050E94062B92
:103A720010F00E940E2BA8950E94BE2411F00C9407
:103A8200861D0E94A8280E94A02A0E94262A0E941F
:103A9200AD2A0E947329CCF50E94D02A0E94D52A11
:103AA2000E94BD2AEA17FB0710F40E94CE2A0E9448
:103AB20073295CF50E94D02A0E94D52A0E94E32A2B
:103AC20020F40E94EB2A319603C00E94EB2A319720
:103AD200FE93EE93A0911C05AA2312F40E94F02AF1
:103AE2000E94F72A14F00E94FF2AA0913605AA2309
:103AF20012F40E942D240E94872914F00E948F291B
:103B02000E94062B10F00E940E2B0E94C32411F07B
:103B12000C94FA1D0E945128129710F40C94FA1D6D
:103B22000E94A8280E94A02A0E94262A0E94AD2A4A
:103B32000E947329CCF50E94D02A0E94D52A0E94A5
:103B4200BD2AEA17FB0710F40E94CE2A0E947329AD
:103B52005CF50E94D02A0E94D52A0E94E32A20F412
:103B62000E94EB2A319603C00E94EB2A3197FE9302
:103B7200EE93A0911C05AA2312F40E94F02A0E943F
:103B8200F72A14F00E94FF2AA0913605AA2312F404
:103B92000E942D240E94872914F00E948F290E94DE
:103BA200062B10F00E940E2B0E94112BD0018827A9
:103BB20099270E94372EA8F40E9434240E942D24B3
:103BC2000E941F240E9426240E946B290E943B29E6
:103BD20055240E943C2A0E943F2A0E943F2A0E94AA
:103BE2004D2A0E94262AED34A4E0FA0710F00E9422
:103BF2006B29E1E0E51511F00C94FB1E062C072859
:103C020089F4A0913205AA236AF40E94172B14F4B6
:103C12000E941D2B0E94D4292CF40E94272B12F4FF
:103C22000E9434240E94B92489F4A0913205AA2367
:103C32006AF40E94172B14F40E941D2B0E94D429AF
:103C42002CF40E94272B12F40E943424062C0728FD
:103C520011F00C947F1E0E94D6280E94F02910F4C5
:103C62000E9434240E94D6280E94F02910F40C9459
:103C72007F1E0E94092ABCF40E940E280E94312B4A
:103C82000E94D6280E94482BEA0FFB1F0E94362969
:103C92000E944D2B20F40E94DB270E9436290E94AD
:103CA200522B0E94572B0E94D929309711F40E945F
:103CB200022A0E94652B20F40E946A2B319603C0CF
:103CC2000E946A2B3197FE93EE93A0911A05AA23C4
:103CD20012F40E946F2B0E94762B14F00E947E2B0E
:103CE200A0913405AA2312F40E9434240E941A28B7
:103CF20031970E94192A14F40E94852B0E94B9243C
:103D0200B9F50E94092A7CF40E940E280E94312BE8
:103D12000E944D2B20F40E94DB270E9436290E942C
:103D2200522B0E94572B0E94D929309711F40E94DE
:103D3200022A0E94652B20F40E946A2B319603C04E
:103D42000E946A2B3197FE93EE93A0911A05AA2343
:103D520012F40E946F2B0E94762B14F00E947E2B8D
:103D62000E941A2831970E94192A14F40E94852B66
:103D72000E94C324A1F50E9456280E94192A34F4F5
:103D82000E945628E0933305F09334050E94112BCC
:103D9200D001882799270E94372EC8F40E94342424
:103DA2000E942D240E941F240E9426240E946B2917
:103DB2000E943B295524A0E2B0E00E9475270E9490
:103DC2003C2A0E943F2A0E943F2A0E944D2A0E94BA
:103DD200262AED34A4E0FA0710F00E946B29E3E0F2
:103DE200F0E06E167F0630F40E94DB27309711F464
:103DF2000E943424E1E0E515F1F50E94B42411F5A6
:103E0200999904C00E948B2B0E948D289A9907C011
:103E12000E948B2BED91FD913197FE93EE93989931
:103E220002C00E94942B9B9902C00E94942BCF99AE
:103E320009C00E949B2BA3E3B5E0ED91FD91319760
:103E4200FE93EE930E94872914F00E948F290E940C
:103E52000D2AA436E0E0BE0714F00E94122AA091B7
:103E62003605AA2312F40E942D24A0913405AA2318
:103E720012F40E9434240E94AD28F301309729F4F1
:103E82000E946D24EDEBF7E023C0E130A0E0FA07D9
:103E920029F40E946D24E7ECF7E01AC0E230A0E0BA
:103EA200FA0729F40E946D24E1EDF7E011C0E33036
:103EB200A0E0FA0729F40E946D24EBEDF7E008C0B8
:103EC200E430A0E0FA0741F40E946D24ECE5F2E050
:103ED200FA93EA930E948B21062C072811F00C9486
:103EE200C91FE42D0E94A32439F40E94A12BE5EE00
:103EF200F7E00E9484244CC0E130A0E0FA0739F4D4
:103F02000E94A12BE0EFF7E00E94842441C0E2303E
:103F1200A0E0FA0739F40E94A12BEBEFF7E00E9430
:103F2200842436C0E330A0E0FA0739F40E94A12BC2
:103F3200E5E0F8E00E9484242BC0E430A0E0FA0718
:103F420039F40E94A12BEFE0F8E00E94842420C003
:103F5200E530A0E0FA0739F40E94A12BE9E1F8E08C
:103F62000E94842415C0E630A0E0FA0739F40E94CA
:103F7200A12BE3E2F8E00E9484240AC0E730A0E02B
:103F8200FA0731F40E94A12BEDE2F8E00E948424AA
:103F92000E94B924F1F4ED2D0E94A32429F40E9479
:103FA200A12BE5EEF7E011C0E130A0E0FA0729F419
:103FB2000E94A12BE0EFF7E008C0E230A0E0FA0790
:103FC20041F40E94A12BEBEFF7E0FA93EA930E94EF
:103FD2008B210E94BE24F1F4E82D0E94A32429F42F
:103FE2000E94A12BE5EEF7E011C0E130A0E0FA0754
:103FF20029F40E94A12BE2EFF7E008C0E230A0E032
:10400200FA0741F40E94A12BEBEFF7E0FA93EA934F
:104012000E948B210E94C32481F5EC2D0E94A324CF
:1040220029F40E94A12BE5EEF7E023C0E130A0E0E5
:10403200FA0729F40E94A12BE2EFF7E01AC0E2305E
:10404200A0E0FA0729F40E94A12BEBEFF7E011C0E0
:10405200E330A0E0FA0729F40E94A12BE5E0F8E0A2
:1040620008C0E430A0E0FA0741F40E94A12BEFE07F
:10407200F8E0FA93EA930E948B210E94AD280E94F5
:104082006028E7E3F8E00E948424A895E0913505D2
:10409200F0913605E0932B05F0932C050E94202A1F
:1040A2000E945D1A8F010E949527EEE4F8E00E94BB
:1040B200842A0E94262A0E9467280E948B2A8CE06A
:1040C2000E94C92360960E9488240E9495270E941C
:1040D2007E210E94C82AA8950E94851AE093450570
:1040E200F09346050E94851A9F010E9425270E948F
:1040F2005D1AE0934305F09344050E949527E2E69A
:10410200F8E0FA93EA93F9010E9467280E945A297B
:10411200F8010E9467288CE00E94C92360960E94E1
:1041220004290E9495270E947E21A8950E94D929E0
:10413200EE0FFF1FE1BFE0913505F0913605EE0F5E
:10414200FF1FE09386000E9449293196E3BDA8959E
:10415200E4E0F0E06E167F0690F49A9B07C00E949E
:104162009B2B0E94BC273196FE93EE93999B07C02E
:104172000E949B2B0E94BC273197FE93EE930E94D4
:10418200B929A233E1E0BE0770F00E94B929AC322E
:10419200E1E0BE0730F4ECE2F1E0E0932105F093B8
:1041A20022050E941F240E94262A339720F40E948F
:1041B2002D240E943424552021F49B9902C0CF9BC8
:1041C200FECF0E94D71AA8950C94891CFFCFFFE05E
:1041D200FA95F1F70895A1B3AF70A1BB919A9098A7
:1041E200F6DF929AF4DFA0B39298F1DF929AEFDFB2
:1041F2009298A7FDF5CF0895A07FAB2BA2BB929A10
:104202000E94E82092980E94E82008959198A1B314
:10421200A76FA1BBB2B3BF70A881EEDFA881A29540
:10422200EBDF919A0C94F523929A0E94E820E0B376
:1042320092980E94E820E07F08950E94E820F4DF2F
:10424200AE2FF2DF9198E295EA2B08950E94EC20BE
:104252000E94A72BEF57FA4FE081F0E0DF01E981DE
:10426200F0E0EA0FFB1FEA930E940721E981E09345
:104272008505E881E0938605229608950E94EC2048
:10428200E2E0EA930E9407210E94EC20ECE0EA932C
:104292000E9407210E94EC20E1E0EA930E9407219C
:1042A200E0E0E0938605E09385050895EF93FF93A0
:1042B200A8816894AA3061F0E894E0918505EF5FE7
:1042C200E0938505E0918705A0918505EA1760F4E2
:1042D200E0918605EF5FE0938605E0E0EA93E091E6
:1042E2008605EA93B3DF2EF076DF909AA881AA932F
:1042F2008DDFFF91EF910C94F5231A93A981BA8176
:10430200ED91A983BA831E2FE03019F01A93CEDF04
:10431200F5CF0EC01A93E981FA813196E983FA83C7
:104322003197E4911E2FE03019F01A93BFDFF3CFDB
:10433200188123960895AA27BB271197F1F70895AC
:104342009198A1B3A76FA1BBB2B3BF70A8810E941D
:10435200FD20919A0C94F52392989098E881E0932D
:1043620087050E94A72BE058FF4FE09383050E9428
:10437200A72BE054FF4FE09384050E94AA2B0E94D2
:10438200AA2B0E94AA2BD7DFE0E2EA93D9DFD3DF80
:10439200EAE20E94B02BE4E00E94B02BE5E80E9422
:1043A200B02BA1B3AF70A1BB919A0E941E21E53040
:1043B20019F0E0E00C94F5230E94EC20E6E0EA9389
:1043C2000E9407210E943F21E1E00C94F5235D9BAE
:1043D200FECFE881ECB908C21A930A93AC81BD8181
:1043E2000E94652C3097C1F0AA81BB810E94652C86
:1043F2008F01309749F00230E0E01E0760F0F801CB
:1044020031978F01ED93FC93AC81BD810E948D2881
:104412003197AE81A08303C0EE81EA93D8DF198180
:1044220008812796089526970E943C2E10E0EA897B
:10443200FB893196EA8BFB8B3197E4912E2FE0308A
:1044420011F40C94C523E12F0E94A32439F42532E0
:1044520011F411E002C00E94B52B95C1E130A0E039
:10446200FA07A9F4253219F40E94B52B8BC112E088
:1044720040E000E02D3211F401E085C12B3211F44D
:104482004BE281C1203211F440E27DC104C0E2302E
:10449200A0E0FA0761F450E013E0203339F40E94FF
:1044A200C02BE0E8F0E0EA2B0E2F6DC106C0E3302E
:1044B200A0E0FA0711F00C94C423203310F02A3341
:1044C20008F015C0A52FB0E0EAE0F0E0EA02F00142
:1044D2005E2F652F7727A22FB0E0E0E3F0E00E9485
:1044E2007D2CEA1BFB0BDB01EA0F5E2F4CC10E9405
:1044F200C32BE336A0E0FA0749F40E94C62BE889F1
:10450200F989A481AA930E94CC2B3CC1E337A0E095
:10451200FA0741F40E94C62B0E94D62B0E94F72371
:104522001E2F11C0E037A0E0FA07D9F40E94C62B73
:104532000E94D62B0E9401241E2F0E94C02BE8E06D
:10454200F0E0EA2B0E2F0E94C02BE2E0F0E0EA2B13
:104552000E2F0E94C02BEFE7FFEFEA230E2F30E071
:104562004FC0E436A0E0FA0721F0E936A0E0FA07EE
:1045720039F40E94C02BE4E0F0E0EA2B0E2F04C0D5
:10458200E537A0E0FA0731F4ECE8F0E0EE83FF83D0
:1045920015E016C0E835A0E0FA0739F40E94C02BF6
:1045A200E8E0F0E0EA2B0E2F06C0E837A0E0FA07B9
:1045B20011F00C94C323E6E9F0E0EE83FF8314E0EC
:1045C2000E94C02B0E94E02BB9F00E94C62B0E94D1
:1045D200E62BAB85AA233AF4EA85FB850E94282CB8
:1045E200EA87FB874DE2403011F01F5F04C00E9452
:1045F200C02B0E94EE2B04C00E94C62B0E94E62B09
:104602000E94F32BE9F41517D8F40E94C02BE0E8BE
:10461200F0E0EA23FB23309771F00E94C02B0E9446
:10462200E02B39F00E94C02B0E94EE2B242F115058
:1046320001C020E301C020E20E94B52B5150E3CF1C
:10464200312F0E94C02BE2E0F0E0EA23FB233097F7
:1046520001F13030E9F00E94C02BE8E0F0E0EA23FB
:10466200FB23309741F0EE81FF813196EE83FF8389
:104672003197E49105C0AE81BF81ED91AE83BF83D6
:10468200EA930E94CC2B503009F051503150E1CFC7
:104692006EC020E3EE81FF810E94692CE887F987D2
:1046A200EE81FF813296EE83FF83E885F985AA8544
:1046B200BB85AE17BF0750F02F5FA885B985EA8585
:1046C200FB85EA1BFB0BEA87FB87EFCF2A3380F0DF
:1046D2000E94C02BE8E0F0E0EA23FB23309721F0B0
:1046E2000E94C32B379603C00E94C32BB7962E2F6E
:1046F2000E94C02BE0E1F0E0EA23FB23309761F552
:10470200213320F4A885B985119709F410C05317F5
:1047120018F00E94F32B09F024C020E20E94C02B63
:10472200E0E8F0E0EA23FB233097B1F020E3A02F8A
:10473200B0E0E0E1F0E0EA2B0E2F0E94C02B0E94D5
:10474200E02B51F00E94C02B0E94EE2B4A930E9454
:10475200CC2B503009F051500E94B52B503009F04B
:1047620051503150A885B985129708F092CF0E9416
:10477200F32B41F0503031F05150E0E2EA930E94C5
:10478200CC2BF8CF10E053CE0E94432E64960895AE
:10479200FF920E94F72BDE0116960E94002CEA83FC
:1047A200FB83DE0114960E94002C0E94052CAA8134
:1047B200BB81E0E0EC930CC0FF920E94F72BE0E09B
:1047C200EA83EB83DE0114960E94002C0E94052CE2
:1047D200198108812496FF900895E881EFB9EEB11E
:1047E200F0E0E078E1F3EFB121960895A991B99153
:1047F200EE27FF276D91662311F03196FBCF0895C6
:10480200AA27BB27E991F9910590002011F0119692
:10481200FBCFFD0108950A921A92FA926A937A9353
:104822008A939A93AA93BA93EA93FA93EFB7EA9385
:104832000895A9E2B1E00E948C2C0895E0E0F0E036
:10484200E0932105F09322050895E0E0F0E0E09383
:104852002305F09324050895E0E0F0E0E0933505A8
:10486200F09336050895E0E0F0E0E0933305F0932D
:1048720034050895AA24BB245524ACE1B0E0E0E05D
:10488200F0E00E94A02CAEE1B0E00E94A02CAC9A15
:10489200E4EFF1E0FA93EA930E94132CAC98E4EF70
:1048A200F1E0FA93EA930E94132CAC9AE4EFF1E060
:1048B200FA93EA930E94132CAC98E4EFF1E0FA9396
:1048C200EA930E94132CAC9AE4EFF1E0FA93EA9394
:1048D2000E94132CAC980895E0E0EA93EA930C94BA
:1048E2002721EEE4F1E0FA93EA930E948B21E0E0C3
:1048F200EA930895E3E0EA930E942721F2CFE1E0F0
:10490200EA930C942721FA93EA930C948B21E0E02A
:10491200EA93E2E0EA930C942721A0E0B0E00E943F
:104922008C2C0895E1500E94A82CEF5F0895EEE1CF
:10493200F0E0FA93EA930C94132CEF5F0E94A82CF8
:10494200E1500895F0E0309708950E943F21E4EF8E
:10495200F1E0FA93EA930C94132CE0E0EA93CACFC5
:10496200EEE4F1E0D0CFE4E0F0E0E615F7050895DB
:10497200E1E0F0E0E615F7050895E2E0F0E0E61583
:10498200F7050895E3E0F0E0E615F7050895E6E897
:10499200F2E0B9CFA4E3B0E00E94882CE0932305B3
:1049A200F0932405A2E3B0E00E94882CE093210555
:1049B200F0932205A0E5B0E00E94882CAEE2B0E0C0
:1049C2000E94A02CA6E5B0E00E94882CA0E1B0E0F5
:1049D2000E94A02CACE5B0E00E94882CAEE0B0E0D2
:1049E2000E94A02C08950E94882CA2E1B0E00E94AF
:1049F200A02C0895A6E3B0E00E94882CA8E0B0E0C5
:104A02000E94A02C08950E94882CAAE0B0E00E9487
:104A1200A02C08950E94882CACE0B0E00E94A02C4B
:104A22000895A5E1B1E00E94882CE0933905F09346
:104A32003A05A5E0B1E008950E94882CE09337057D
:104A4200F09338050895EBE9F2E05DCFAEE3B0E014
:104A52000E94882CE0932305F0932405ACE3B0E098
:104A62000E94882CE0932105F0932205A2E5B0E094
:104A72000E94882CAEE2B0E00E94A02CA8E5B0E033
:104A82000E94882CA0E1B0E00E94A02CAEE5B0E02C
:104A92000E94882CAEE0B0E00E94A02C0895A0E411
:104AA200B0E00E94882CA8E0B0E00E94A02C0895FB
:104AB200A7E1B1E00E94882CE0933905F0933A0512
:104AC200A7E0B1E00895E0EBF2E01DCFA8E4B0E08A
:104AD2000E94882CE0932305F0932405A6E4B0E01D
:104AE2000E94882CE0932105F0932205A4E5B0E012
:104AF2000E94882CAEE2B0E00E94A02CAAE5B0E0B1
:104B02000E94882CA0E1B0E00E94A02CA0E6B0E0B8
:104B12000E94882CAEE0B0E00E94A02C0895AAE486
:104B2200B0E00E94882CA8E0B0E00E94A02C08957A
:104B3200A9E1B1E00E94882CE0933905F0933A058F
:104B4200A9E0B1E00895AAE6B0E00E94882CE093C3
:104B52002305F0932405A8E6B0E00E94882CE09398
:104B62002105F0932205ACE6B0E00E94882CAEE26B
:104B7200B0E00E94A02CAEE6B0E00E94882CA0E13A
:104B8200B0E00E94A02CA0E7B0E00E94882CAEE02A
:104B9200B0E00E94A02C0895A4E7B0E00E94882C07
:104BA200A8E0B0E00E94A02C0895ABE1B1E00E9421
:104BB200882CE0933905F0933A05ABE0B1E0089513
:104BC200ACE7B0E00E94882CE0932305F093240523
:104BD200AAE7B0E00E94882CE0932105F093220519
:104BE200AEE7B0E00E94882CAEE2B0E00E94A02CBA
:104BF200A0E8B0E00E94882CA0E1B0E00E94A02CC6
:104C0200A2E8B0E00E94882CAEE0B0E00E94A02CA6
:104C12000895A6E8B0E00E94882CA8E0B0E00E94C7
:104C2200A02C0895ADE1B1E00E94882CE0933905F3
:104C3200F0933A05ADE0B1E00895AEE8B0E00E942D
:104C4200882CE0932305F0932405ACE8B0E00E94A1
:104C5200882CE0932105F0932205A0E9B0E00E94A0
:104C6200882CAEE2B0E00E94A02CA2E9B0E00E9443
:104C7200882CA0E1B0E00E94A02CA4E9B0E00E9440
:104C8200882CAEE0B0E00E94A02C0895A8E9B0E024
:104C92000E94882CA8E0B0E00E94A02C0895AFE109
:104CA200B1E00E94882CE0933905F0933A05AFE019
:104CB200B1E00895A0EAB0E00E94882CE0932305B9
:104CC200F0932405AEE9B0E00E94882CE093210520
:104CD200F0932205A2EAB0E00E94882CAEE2B0E096
:104CE2000E94A02CA4EAB0E00E94882CA0E1B0E0CF
:104CF2000E94A02CA6EAB0E00E94882CAEE0B0E0B0
:104D02000E94A02C0895AAEAB0E00E94882CA8E094
:104D1200B0E00E94A02C0895A1E2B1E00E94882C8C
:104D2200E0933905F0933A05A1E1B1E00895A2EBD1
:104D3200B0E00E94882CE0932305F0932405A0EBB9
:104D4200B0E00E94882CE0932105F0932205A4EBA9
:104D5200B0E00E94882CAEE2B0E00E94A02CA6EB4C
:104D6200B0E00E94882CA0E1B0E00E94A02CA8EB49
:104D7200B0E00E94882CAEE0B0E00E94A02C089522
:104D8200ACEBB0E00E94882CA8E0B0E00E94A02C1E
:104D92000895A3E2B1E00E94882CE0933905F093D4
:104DA2003A05A3E1B1E00895E4EFF1E0FA93EA9362
:104DB2000E94132C0C943F21A2ECB0E00E94882C9C
:104DC200E0932305F0932405A5ECB0E00E94882C23
:104DD200AEE2B0E00E94A02CA7ECB0E008950E94E1
:104DE200882CAEE0B0E00E94A02C08950E948C2C8A
:104DF200A2E1B0E0F0E00E94A02C0895A9ECB0E09E
:104E02000E94882CE0932305F0932405ACECB0E0DB
:104E12000E94882CAEE2B0E00E94A02CAEECB0E082
:104E22000895A0EDB0E00E94882CE0932305F09352
:104E32002405A3EDB0E00E94882CAEE2B0E00E940F
:104E4200A02CA5EDB0E00895E8ECF0E0FA93EA9327
:104E52000C94132CA7EDB0E00E94882CE09321055E
:104E6200F0932205A9EDB0E008950E94882CA0E1FC
:104E7200B0E00E94A02C08950E94882CE0932105A6
:104E8200F09322050895A5EEB0E00E94882CE093ED
:104E92002305F0932405A7EEB0E0A1CF0E94882C51
:104EA200A3EEB0E00E94A02C08950E94882CE0930B
:104EB2002305F09324050895EDE6F3E024CDEBE419
:104EC200F5E0FA93EA930C947E21A6E0B0E00E940A
:104ED200882C089531970E94A02C3196089531961E
:104EE2000E94A02C31970895E0E0F0E00E94A02CEF
:104EF2000895659785E1A0E0B0E00895FE01FA9378
:104F0200EA930E947E2165960895A1E0B0E00E9496
:104F12008C2C0895A2E0B0E00E948C2C0895A3E0AE
:104F2200B0E00E948C2C0895E0E0F5E0FA93EA9359
:104F32000895E2E8F3E0FA93EA93E0912105F09113
:104F42002205662777270E946D2C84E00E94C923E0
:104F52002896E2E0EA93E3E0EA930E942721E4CF75
:104F62000E947E21E0E0EA93CACCE1E9F3E0CBCCF7
:104F7200E6EAF3E0C8CCA1E2B5E0ED91FD91089537
:104F82003197FE93EE93E2E3F0E0FA93EA930C9406
:104F9200132C3196FE93EE93E2E3F0E0FA93EA9358
:104FA2000C94132CA0912105B0912205AD32E1E0C1
:104FB200BE070895E0912105F09122050895E2E8E7
:104FC200F3E0FA93EA930895A3E0B1E00E94882CFB
:104FD2000895662777270E946D2C84E00E94C923DA
:104FE2002896E2E0EA93E3E0EA930E9427219CCF2D
:104FF200E2E3F0E0FA93EA930C94132CEBEBF3E088
:10500200FA93EA93A0E1B0E00E94882CE2CFEFECA1
:10501200F3E079CCE4EEF3E076CCA0E1B0E00E94DC
:10502200882C0895A0E1B0E0EFE0F0E00E94A02C0F
:105032000895E0913705F091380508950E94402CBB
:105042000E946D2C84E00E94C9232896E2E0EA9334
:10505200E3E0EA930E94272167CFED91FD9190CF83
:10506200ED91FD9196CFE4E6F0E0E0933705F09301
:1050720038050895E0912305F09124050895E9E1AA
:10508200F4E041CCA3E2B5E0E8CFA3E2B5E0E8CF9B
:10509200A0912305B0912405AB3EE1E0BE0708953F
:1050A200A0912305B09124050895A3EEB0E00E94DB
:1050B200882C0895E4E6F0E00E94A02C0895E0E038
:1050C200EA931DCCE3E0EA930C9427216627772725
:1050D2000E946D2C089588E00E94C9232C960895A1
:1050E200A6E1B0E00E94842C0895ED91FD913197E4
:1050F200FE93EE93F5CFE130A0E0FA07A0E06A0755
:10510200A0E07A070895A6E1B0E0E0E0F0E060E018
:1051120070E00E94982C0895ED91FD913196FE93D6
:10512200EE930895A6E1B0E00E94982CADE1B5E0BF
:105132000895E0931D05F0931E050895EBEBF3E04F
:10514200FA93EA93AEE0B0E00E94882C42CFAEE040
:10515200B0E00E94882C0895E4E6F0E0FA93EA9326
:105162000C94132CAEE0B0E0EFE0F0E00E94A02C33
:105172000895E0913905F0913A050895E4E6F0E0EA
:10518200E0933905F0933A050895E6EBF4E0FA93DB
:10519200EA93AEE2B0E00E94882C98CF84E00E94AD
:1051A200C9232896E0E0EA938DCFAEE2B0E00E94F8
:1051B200882C0895A2E1B0E00E94882C0895A2E113
:1051C200B0E092CEE5E0F5E09ECBEAE1F5E09BCBE4
:1051D200A2E1B0E00E948C2C0895A8E0B0E00E9409
:1051E200882C0895A4E0B0E0E1E0F0E00E94A02C59
:1051F2000895AAE0B0E00E94882C0895ACE0B0E0E7
:105202000E94882C0895E0E0EA935CCFAAE2B0E025
:105212000E94882C089584E00E94C923289677CBA7
:10522200ACE2B0E00E94882C0895A4E1B0E00E94B4
:10523200882C0895E2ECF1E00E94A02C0895E1E0B0
:10524200F0E00E94A02C0895E6E1F0E00E94A02C7C
:105252000895EFE0F0E00E94A02C0895E0E0F0E075
:10526200E0931105F09312050895E0931705F0936A
:1052720018050895ACE1B0E037CEE0E0F0E0E0934D
:105282001905F0931A05E0931B05F0931C05089588
:10529200A7E2B1E00E94882C0895E2E6F6E033CB63
:1052A200E7E7F6E030CBEBE8F6E0FA93EA93E2DEEA
:1052B2000DCF80DE0BCF0E947E21E1E05E2EAA247C
:1052C200BB24D8CFE5E9F6E0FA93EA93F2CFA0E364
:1052D200B0E00ACEAAE1B0E007CEA0914505B091B8
:1052E20046050895A0912D05B0912E050E94332EFA
:1052F2000895E0913505F09136053F97E093350525
:10530200F0933605A0913605AA230895A09135059C
:10531200B0913605A436E0E0BE070895E4E6F0E079
:10532200E0933505F09336050895E0914505F09137
:10533200460508959FDED1DFAE17BF070895A0E2AC
:10534200B0E00E94882CCBCDE0914305F09144055A
:105352000895A0914305B09144050895A0913105A7
:10536200B09132050895E0914705F09148050895FE
:10537200A0912105B09122050895AE0FBF1FEAE06A
:10538200F0E00E944A2CDF01E3E2F0E00E94522C9E
:10539200E0933305F0933405E6DF3A96E093470550
:1053A200F09348050895DADFAD3FEFEFBE070895A9
:1053B200E0913305F091340508957497E093330535
:1053C200F0933405A0913405AA230895C2DFEA17A9
:1053D200FB070895ACE1B0E00E94882C80CDB9DFD4
:1053E200AE17BF070895A0E3B0E00E94882C08958D
:1053F200AC9AE0E9F1E0FA93EA930E94132CAC989C
:105402000895E3E2F0E0E0933305F0933405089564
:10541200A5DF0E94332E0895A0913305B091340583
:105422000895E4E6F0E0E0933305F093340508953F
:10543200F3DFEA17FB070895A3E3B5E06DCEB8DF0B
:10544200E0932905F0932A050895AAE1B0E00E94AD
:10545200882C08956ADFE0932305F09324050895CC
:10546200E0E9F1E0FA93EA930C94132CA4E6B0E09D
:105472000E944A2C0895AA24BB2429CFAC9AE4EFB7
:10548200F1E0FA93EA930E94132CAC98E4EFF1E076
:10549200FA93EA930C94132CAC9AE4EFF1E0FA93AA
:1054A200EA930E94132CAC980895E3E5EDB9E0E08D
:1054B200EEB9B99ABA9ABB980895E0E0EA930E94CD
:1054C200EE23F0E0089566277727DF01CB01E8E0BD
:1054D2000E94342C0895662777270E94232C8F017F
:1054E200087F1F77169507951695079516950795C8
:1054F20008950E94402C0E941F2D089584E00E946E
:10550200DD2326960895FA93EA93E0912B05F09114
:105512002C05DCCDE0912905F0912A05D7CDFA932F
:10552200EA9380E00E94DD2322960895EAE4F7E000
:10553200F6CFE8E5F7E0F3CFE1E6F7E0F0CFDF0101
:10554200EAE0F0E00E94522CD4DFA3E1B5E00E9431
:10555200E62CED93FC930895A0911305B0911405E8
:105562000E944A2CE0931105F09312050895A4E0DD
:10557200B0E00E94882C08957DDDA0911105B091C4
:1055820012050895E0931105F09312050895ECE2D7
:10559200F1E0FA93EA930C94132C6CDDF3CFE091D3
:1055A2001105F091120562CFDF01E0911B05F09128
:1055B2001C05E650FF4F0E94522CE0933505F093F4
:1055C20036050895B2DEA0911105B0911205AE170D
:1055D200BF070895ABE1B5E0ED91FD910895E0E0DC
:1055E200F0E0E0931B05F0931C050895A0911B05C4
:1055F200B0911C05AD32E1E0BE070895ECE2F1E0A6
:10560200E0931B05F0931C050895A0911105B0913C
:105612001205A33CE1E0BE070895E2ECF1E0B2CF4F
:10562200A0E2B0E00E94882C0F015ACD97DEEDEF88
:10563200FFEFEA17FB0708959BDEE5E0F0E00E942A
:10564200522CE0933305F09334050895B1DE7E9732
:10565200E0933305F0933405A0913405AA2308950D
:10566200DF01EAE0F0E00E94522C43DFA5E1B5E061
:105672000E94E62CED93FC93ACE1B0E00E94882CF2
:10568200A0911505B09116050E944A2CEECDA0916D
:105692001705B091180508958DDCF9DFEA17FB07AD
:1056A2000895E0911705F0911805E0CEDF01E09131
:1056B2001905F0911A05EA56FF4F0E94522CE09309
:1056C2003305F093340508953FDEE1DFAE17BF07DF
:1056D2000895A9E1B5E0ED91FD910895E0E0F0E0D3
:1056E200E0931905F0931A050895A0911905B09158
:1056F2001A05AD32E1E0BE070895ECE2F1E0E09375
:105702001905F0931A05089594DCE0933305F0939C
:1057120034050895E9E1F0E0FA93EA930E94132C2C
:10572200A5E3B5E00895E9E1F0E0FA93EA930E9477
:10573200132C82CEE9E1F0E0FA93EA930C94132C55
:10574200EAE0EA93E0E0EA930C942721E881F0E0B2
:1057520008950E949C21E0E3EA930C94A121EA932C
:105762000E9407210C949C212A93EF85F889FA93D1
:10577200EA93FE013F96FA93EA930C94ED21A02F4F
:10578200B0E00895E22FF0E00895E889F9893497AE
:10579200E88BF98B0895EF85F889FA93EA93FE0175
:1057A2003F96FA93EA930C94ED21A889B98914964D
:1057B2000E94652CEE83FF83FA93EA930895E4E056
:1057C200F0E0EA23FB2330970895A889B98914965B
:1057D2000E94652CEA87FB870895EBEFFFEFEA232F
:1057E2000E2F0895E02FF0E0E1700895F82E229731
:1057F2001A930A93DE010E941F2C8D0108950E94C4
:105802001F2C0E94652C0895FA93EA931A930A9327
:10581200FE013696FA93EA93E0E0F0E0FA93EA9317
:105822000C941422E991F991309639F080ED97E0C9
:105832000197F1F7A8953197C9F708950024AF0DA4
:10584200B01D0895EA2BFB2B682B792B0895F19557
:10585200E195F0400895F09560957095E195FF4FC0
:105862006F4F7F4F0895EE230E2EFD01BC0131F0E4
:10587200EE0FFF1F661F771F0A94D1F708956F2F4F
:10588200660F660B762F08958B2F880F880B982F43
:105892000895FA9FF02DEB9FF00DEA9FE02DF10D98
:1058A20008950024112490E1AA0FBB1F001C111CB3
:1058B2000E1A1F0A18F40E0E1F1E01C0A1609A953F
:1058C20099F7FD01D0010895ED91FC91119708958A
:1058D2000590F491E02D08957A936A93FA93EA93EE
:1058E2000895689401C0E89401D0A9D0182E862F9B
:1058F200612D192E972F712D1B2EBF2FF12D1A2ED0
:10590200AE2FE12D0895129602D0BF011297119683
:1059120002D0FE2F1197E199FECFFF93FFB7F894C3
:10592200AEBBBFBBE09AEDB3FFBFFF91089507D0B6
:1059320012960F01FB0103D0F0011297089507D0D0
:105942001196EF93EF2F03D0EF9111970895E19BFA
:1059520002C0A895FCCF9FB7F894AEBBBFBBE09A3C
:105962008DB3E81719F0EDBBE29AE19A9FBF089553
:10597200552342F4503811F4E0FF04C03196691FF8
:10598200791F6BF050E8572711F45F93C6C05F3F51
:1059920031F0660F000C57956795752F08955F9348
:1059A20000200AF0C6C0BFC050E8192E1522880F89
:1059B200991F9527550F879550E8072E0522660FE8
:1059C200771F7527550F67950895689401C0E8946D
:1059D2005F93F2DF703818F07F3F08F49EC056E103
:1059E200571BAAF4519558300EF4593030F0EFEFAE
:1059F200FFEF6FEF7FE777F91AC077275523B9F0EA
:105A0200EE0FFF1F661F771F5A95D1F710C0772739
:105A1200583028F0EF2FF62F672F5850F9CF552323
:105A220031F076956795F795E7955A95D1F700206D
:105A32000AF411DF5F910895689401C0E8943097E9
:105A420060407040B1F0002426F0772312F40094F5
:105A520002DF172E7EE1112032F07A95EE0FFF1F42
:105A6200661F111CF9CFEF2FF62F612D5F938ADF8E
:105A72005F9108954F93AF01FD01DA01AB01BC01C3
:105A8200CA01402D012C142E4F910895EA0FFB1FDD
:105A9200681F0895E095F0956095EF5FFF4F6F4F97
:105AA20008955F9381DF903839F1703821F1572FD3
:105AB200591B13F112F4DEDFFACF583118F0AA277E
:105AC200BB278827583028F0AB2FB82F882758508B
:105AD200F9CF552329F08695B795A7955A95D9F709
:105AE200502D512562F0D2DF38F46795F795E7958E
:105AF200739513F41EC0BEDF45DF5F910895EA1B64
:105B0200FB0B680B51F010F40094C4DF6623A2F380
:105B1200EE0FFF1F661F7A95CBF7EE27FF2766274A
:105B220077275F910895EFEFFFEF6FE77FEF5F91C8
:105B32000895EFEFFFEF6FE77FE75F9108955F93BF
:105B420033DF703851F3903841F301240894791F00
:105B520023F41CF300203AF3ECCF0F921F932F9300
:105B62003F934F93112722279927689FA0018F9F68
:105B7200302D410D591F6B9F300D411D591F8E9FB6
:105B820027D0BF9F25D06A9F23D0BE9F1DD0AF9F35
:105B92001BD0AE9F110D291F391F491F591FE32F1B
:105BA200F42F652F522F4F913F912F911F910F90FC
:105BB20066232AF0550FEE1FFF1F661F02C0739562
:105BC2004BF2D6DE5F910895100D211D391F02C0E0
:105BD200200D311D491F591F08955F93E5DE70386E
:105BE20021F411200AF49FCFA4CF903809F495CF65
:105BF20001240894970B1BF4D4F30020F3CF792FE0
:105C02001F932F933F934F9311241127222733275A
:105C12004427552790E2AE17BF078607410730F0A9
:105C2200AE1BBF0B860B410B089401C08894551F15
:105C3200221F331F111CAA1FBB1F881F441F9A95C6
:105C420051F7F901612D4F913F912F911F916623D9
:105C520032F0550FEE1FFF1F661F7A9543F288DE62
:105C62005F91089500240A160B060895EA17FB07B0
:105C72006807790708955A934A933A932A931A9395
:105C82000A9308955D814C813B812A8119810881A3
:105C92000895AC0FBD1F05900D928A95E1F7089506
:00000001FF
